:020000040800F2
:10000000A00C002011020008E5070008C702000844
:10001000E1070008C10200082109000800000000F3
:10002000000000000000000000000000E9070008D8
:10003000C502000800000000E7070008EB07000801
:100040002B0200082B0200082B0200082B020008DC
:100050002B0200082B0200082B0200082B020008CC
:100060002B0200082B0200082B0200082B020008BC
:100070002B0200082B0200082B0200082B020008AC
:100080002B0200082B0200082B0200082B0200089C
:100090002B0200082B0200082B0200082B0200088C
:1000A0002B0200082B0200082B0200082B0200087C
:1000B0002B0200082B0200082B0200082B0200086C
:1000C0002B0200082B0200082B0200082B0200085C
:1000D0002B020008710800082B0200082B02000800
:1000E0002B0200082B0200082B0200082B0200083C
:1000F0002B0200082B0200082B0200082B0200082C
:100100002B0200082B0200082B0200082B0200081B
:100110002B0200082B0200082B0200082B0200080B
:100120002B0200082B0200082B0200082B020008FB
:1001300000F002F800F05CF80AA090E8000C82449D
:100140008344AAF10107DA4501D100F051F8AFF27A
:10015000090EBAE80F0013F0010F18BFFB1A43F0A5
:1001600001031847C4110000E41100000A444FF0D5
:10017000000C10F8013B13F0070408BF10F8014B06
:100180001D1108BF10F8015B641E05D010F8016B4B
:10019000641E01F8016BF9D113F0080F1EBF10F8AF
:1001A000014BAD1C0C1B09D16D1E58BF01F801CBD2
:1001B000FAD505E014F8016B01F8016B6D1EF9D555
:1001C0009142D6D37047000000230024002500266A
:1001D000103A28BF78C1FBD8520728BF30C148BFAA
:1001E0000B6070471FB500F0A1FD1FBD10B510BD1D
:1001F00000F033F81146FFF7F5FF00F04BFC00F07C
:1002000051F803B4FFF7F2FF03BC00F08BFB0000D2
:100210000948804709480047FEE7FEE7FEE7FEE79A
:10022000FEE7FEE7FEE7FEE7FEE7FEE704480549D6
:10023000054A064B70470000F50700083101000829
:10024000A0040020A00C0020A0080020A00800208E
:1002500070477047704770477047754600F02CF83C
:10026000AE4605006946534620F00700854618B0A3
:1002700020B5FFF7DBFFBDE820404FF000064FF050
:1002800000074FF000084FF0000B21F00701AC46CB
:10029000ACE8C009ACE8C009ACE8C009ACE8C009EA
:1002A0008D46704710B50446AFF300802046BDE888
:1002B0001040FFF7A6BF0000004870474004002030
:1002C00000BFFEE7704700BFFEE72DE9F04107469B
:1002D0000C4615461E462A2000F02CF9384600F040
:1002E0000BF9284600F008F92B2000F023F92046EE
:1002F00000F002F9304600F0FFF82C2000F01AF967
:10030000BDE8F08170B50646EF231A460021084685
:10031000FFF7DBFF00240AE0002504E0304600F090
:10032000EBF8681C85B2F02DF8DB601C84B2F02C71
:10033000F2DB70BD70B504460D4616462B462246CC
:1003400029462046FFF7C1FF304600F0D5F870BDC2
:100350002DE9F84F05460F4616469A46DDF828B0B7
:100360000095E02D01DCE02F01DDBDE8F88FA6F15E
:100370002000C6B207F10F0083B2E81D82B23946F1
:100380002846FFF7A2FFBAF1000F27D1002422E090
:1003900004EB0610234911F800904FF0000812E01A
:1003A00009F0010018B1584600F0A6F803E01E4815
:1003B000008800F0A1F84FEA6909681C85B208F1CD
:1003C000010000F0FF08B8F1080FE9DB009D781C80
:1003D00087B2601CC4B2102CDADB21E000241DE0DF
:1003E00004EB06100F4911F800904FF0000810E0E0
:1003F00009F0010038B13A1991B205EB080290B248
:100400005A46FFF797FF4FEA690908F1010000F02B
:10041000FF08B8F1080FEBDB601CC4B2102CDFDB67
:1004200000BFA2E7360D0008680300202DE9F84F51
:1004300006468A4690461D46DDF828904FF0000B90
:10044000002431E0281B401EC1B20A2000F082FBCC
:10045000B8FBF0F00A21B0FBF1F201FB1207BBF18F
:10046000000F11D1681EA0420EDD5FB9082101FB0B
:10047000046188B2002320225146CDF80090FFF796
:1004800067FF0FE04FF0010B07F13001CAB20821FE
:1004900001FB046188B200235146CDF80090FFF7BC
:1004A00057FF00BF601CC4B2AC42CBDBBDE8F88F85
:1004B000F8B505460E4614461F4619E0E02D03DD4B
:1004C000002506F1100086B2E02E06DD002005466C
:1004D00006464FF47840FFF715FF00972278002377
:1004E00031462846FFF734FF05F1080085B2641C49
:1004F00020780028E2D1F8BD10B504464FF4807191
:10050000044800F067FA201200F022F8E0B200F090
:100510001FF810BD0008014010B504464FF480716B
:10052000034800F057FA204600F012F810BD000012
:100530000008014010B504464FF48071034800F0F4
:1005400047FA204600F004F810BD00000008014002
:1005500070B504464FF48051124800F039FA002576
:1005600017E020210F4800F033FA04F0800020B19A
:1005700080210C4800F02EFA03E08021094800F0A9
:1005800027FA2021074800F025FA6006040E681CAF
:10059000C5B2082DE5DB4FF48051024800F01AFA8D
:1005A00070BD00000008014010B540F2026000F08C
:1005B000DDFA40F2056000F0D9FA20230322102171
:1005C000854800F009FA802303221021824800F0B8
:1005D00003FA4FF48073032210217F4800F0FCF9E6
:1005E0004FF40063032210217B4800F0F5F94FF42B
:1005F000805303221021784800F0EEF904230322EF
:100600001021764800F0E8F90421744800F0E2F97E
:100610008021714800F0DEF94FF480716E4800F0DF
:10062000D9F94FF400616C4800F0D4F94FF48051CF
:10063000694800F0CFF92021674800F0CBF94FF46A
:100640000061654800F0C4F9C82000F09DF94FF43E
:100650000061614800F0BEF9C82000F095F904215E
:100660005E4800F0B7F9C82000F08EF93620FFF799
:1006700061FF0020FFF750FF3A20FFF75BFF0520E6
:10068000FFF74AFFB220FFF755FF0C20FFF744FFAA
:100690000C20FFF741FF0020FFF73EFF3320FFF75C
:1006A0003BFF3320FFF738FFB720FFF743FF35202C
:1006B000FFF732FFBB20FFF73DFF1920FFF72CFFAC
:1006C000C020FFF737FF2C20FFF726FFC220FFF7DF
:1006D00031FF0120FFF720FFC320FFF72BFF12207F
:1006E000FFF71AFFC420FFF725FF2020FFF714FFB4
:1006F000C620FFF71FFF0F20FFF70EFFD020FFF7E8
:1007000019FFA420FFF708FFA120FFF705FFE02055
:10071000FFF710FFD020FFF7FFFE0420FFF7FCFEDD
:100720000D20FFF7F9FE1120FFF7F6FE1320FFF76B
:10073000F3FE2B20FFF7F0FE3F20FFF7EDFE5420E5
:10074000FFF7EAFE4C20FFF7E7FE1820FFF7E4FE74
:100750000D20FFF7E1FE0B20FFF7DEFE1F20FFF765
:10076000DBFE2320FFF7D8FEE120FFF7E3FED020D9
:10077000FFF7D2FE0420FFF7CFFE0C20FFF7CCFEE0
:100780001120FFF7C9FE1320FFF7C6FE2C20FFF74C
:10079000C3FE3F20FFF7C0FE4420FFF7BDFE5120FF
:1007A000FFF7BAFE2F20FFF7B7FE1F20FFF7B4FEBA
:1007B0001F20FFF7B1FE2020FFF7AEFE2320FFF73A
:1007C000ABFE2120FFF7B6FE1120FFF7B3FE292074
:1007D000FFF7B0FE10BD000000080140001401400A
:1007E00000BFFEE770477047704710B500F09EF8F5
:1007F00010BD000008B51B48006840F4700019499E
:1008000008601948006840F0010017490860084670
:10081000406840F0800048600020009002E00098AE
:10082000401C009044F6206100988842F7D30E489F
:10083000406820F003000C494860084600680B49F6
:100840000840094908604FF41F00886008460068A6
:1008500020F48020086000204860C86200F020FA80
:1008600008BD000088ED00E000100240FFFFF6FE2A
:1008700010B52649264800F03DFA002844D0234907
:10088000234800F02AFA2520002807DB00F01F0289
:10089000012191401F4A430942F8231000BF1C4820
:1008A00000F016FAC4B21C48008800F4004088B971
:1008B0001948008800F4804030B30A2C03D000208F
:1008C0001549088020E01448008840F4004012498F
:1008D000088019E00D2C06D10F48008840F48040B4
:1008E0000D49088010E00C480088C0F30D000B494A
:1008F0000C5409480088401C0749088008460088B5
:10090000C72801DD0020088010BD00000503050098
:100910000038014080E200E07403002078030020EA
:1009200000BFFEE7014600BF7047000004480068B2
:1009300020B103480068401E01490860704700006C
:100940000400002010B56FF0040000F0ADF90A4873
:1009500000680A49B0FBF1F00949087008460078C0
:1009600000EB4001C1EBC0104FF6FF7101EAC0007F
:100970000449088010BD00000000002000127A0029
:100980006A0300206C0300200146104A12884A4383
:100990004FF0E0235A6100229A6101221A6100BFE0
:1009A0004FF0E022106900F001021AB100F4803229
:1009B000002AF5D04FF0E022126922F001024FF038
:1009C000E0231A6100229A61704700006C03002046
:1009D0004161704701617047F0B504461646002535
:1009E000002201F00F0501F0100747B1042E05D1D8
:1009F00045F00305E76B1F43E76300E03543002044
:100A00001EE0012787401F40C7B122684FEA800CD3
:100A10000F2707FA0CF7BA43870005FA07F73A439E
:100A2000282904D1012787401F40676105E0482934
:100A300003D1012787401F4027612260471CB8B2BD
:100A40000828DED3082022E0012787401F40E7B1B5
:100A50006268A0F108074FEA870C0F2707FA0CF726
:100A6000BA43A0F10807BF0005FA07F73A4328295F
:100A700004D1012787401F40676105E0482903D161
:100A8000012787401F4027616260471CB8B21028C9
:100A9000DAD3F0BD08B5FFF755FFFFF785FD40F24B
:100AA000026000F063F80123032210211E48FFF7C3
:100AB00093FF01211C48FFF78BFF34E001211A4806
:100AC000FFF786FFC820FFF75FFF01211648FFF7F9
:100AD00081FFC820FFF758FF4FF4784313A223216A
:100AE0000A20FFF7E5FC4FF4784316A237210A20CD
:100AF000FFF7DEFC4FF478400323F022372100900B
:100B00004620FFF793FC4FF4784310A237216E2064
:100B1000FFF7CEFC4FF478400323F02237210090FA
:100B2000A020FFF783FCC9E700080140312E3534CF
:100B30002054465420535049203234302A32343025
:100B4000000000004C43445F573A00004C43445FB0
:100B5000483A000010B50246012000E050430B1E49
:100B6000A1F10104E1B2F9D110BD0000064A02EB87
:100B70009011096800F01F0301229A401143024BB3
:100B800003EB90121160704700100240002000211A
:100B90003F4A126842F480323D4B1A6000BF401C4D
:100BA0003B4A126802F4003119B94FF6FF729042C5
:100BB000F5D1374A126802F400320AB900BFFEE7E5
:100BC000334AD26942F08052314BDA61314A1268BD
:100BD00042F440422F4B1A602D4A52682C4B5A6007
:100BE0001A4652685A601A46526842F480625A6045
:100BF0001A46526822F440325A601A46526842F449
:100C000040325A601A465268234B1A40204B5A60B1
:100C10001A465268214B1A431D4B5A601A461268F5
:100C200042F080721A6000BF194A126802F0007226
:100C3000002AF9D0174A126842F48032154B1A6024
:100C400000BF144A526802F48032002AF9D0114AD7
:100C5000126842F400320F4B1A6000BF0D4A52680E
:100C600002F40032002AF9D0094A526822F0030245
:100C7000074B5A601A46526842F002025A6000BF9F
:100C8000034A526802F00802002AF9D070470000B7
:100C90000010024000700040FFFFC3B7000034089E
:100CA00010B5FFF773FF10BD042808D14FF0E02105
:100CB000096941F004014FF0E022116107E04FF0B3
:100CC000E021096921F004014FF0E0221161704731
:100CD00001464868C0F30800704710B500EB915218
:100CE0001268C1F304440123A3409A4300EB9153DB
:100CF0001A6010BD70B5024600230024C1F38910AC
:100D0000105801F01F060125B54000EA050302EB6B
:100D100091500068C1F304460125B54000EA05047E
:100D200014B10BB1012070BD0020FCE74FF0407002
:100D3000E1EE100A70470000000000000000000013
:100D4000000000000000000000080808080808086B
:100D500000001818000000486C2412000000000079
:100D60000000000000000000002424247F12121262
:100D70007F12121200000000081C2A2A0A0C1828F0
:100D8000282A2A1C080800000022251515152A58B3
:100D90005454542200000000000C1212120A76254E
:100DA0002911916E000000060604030000000000F7
:100DB000000000000000004020101008080808088B
:100DC0000810102040000002040808101010101035
:100DD0001008080402000000000008086B1C1C6BCF
:100DE00008080000000000000000080808087F084C
:100DF00008080800000000000000000000000000DB
:100E00000000060604030000000000000000FE00D1
:100E100000000000000000000000000000000000D2
:100E2000000006060000000080404020201010084E
:100E30000804040202000000001824424242424218
:100E4000424224180000000000080E0808080808A4
:100E50000808083E00000000003C424242202010EA
:100E60000804427E00000000003C4242201820405E
:100E70004042221C000000000020302824242222AE
:100E80007E20207800000000007E0202021A264028
:100E90004042221C0000000000382402021A2642B0
:100EA0004242241800000000007E22221010080890
:100EB0000808080800000000003C424242241824B0
:100EC0004242423C00000000001824424242645862
:100ED0004040241C00000000000000001818000022
:100EE00000001818000000000000000000080000CA
:100EF000000000080804000000402010080402045C
:100F00000810204000000000000000007F000000EA
:100F10007F000000000000000002040810204020B4
:100F20001008040200000000003C4242464020102D
:100F30001000181800000000001C225A5555555585
:100F40002D42221C00000000000808181414243C44
:100F5000224242E700000000001F2222221E2242FD
:100F60004242221F00000000007C424201010101B8
:100F70000142221C00000000001F22424242424265
:100F80004242221F00000000003F4212121E1212B5
:100F90000242423F00000000003F4212121E1212A5
:100FA0000202020700000000003C22220101017140
:100FB0002122221C0000000000E7424242427E4201
:100FC000424242E700000000003E08080808080806
:100FD0000808083E00000000007C101010101010DF
:100FE00010101010110F0000007722120A0E0A12C2
:100FF0001222227700000000000702020202020211
:101000000202427F000000000077363636362A2A78
:101010002A2A2A6B0000000000E346464A4A525240
:101020005262624700000000001C224141414141E0
:101030004141221C00000000003F424242423E0269
:101040000202020700000000001C22414141414110
:101050004D53321C60000000003F4242423E1212DB
:10106000222242C700000000007C424202041820F5
:101070004042423E00000000007F4908080808087E
:101080000808081C0000000000E7424242424242B9
:101090004242423C0000000000E742422224241465
:1010A0001418080800000000006B494949495555CB
:1010B000362222220000000000E7422424181818DB
:1010C000242442E7000000000077222214140808BC
:1010D0000808081C00000000007E212010100804F1
:1010E0000442423F00000078080808080808080881
:1010F0000808080878000000020204040808081024
:10110000102020204040001E101010101010101051
:10111000101010101E0000384400000000000000F5
:1011200000000000000000000000000000000000BF
:101130000000000000FF00060800000000000000A2
:10114000000000000000000000000000003C4278A9
:10115000444242FC0000000000030202021A264240
:101160004242261A0000000000000000003844023D
:1011700002024438000000000060404040784442D1
:10118000424264D80000000000000000003C427EA3
:101190000202423C0000000000F08808087E0808B7
:1011A0000808083E0000000000000000007C222229
:1011B0001C023C42423C000000030202023A46424A
:1011C000424242E700000000000C0C00000E08083C
:1011D0000808083E000000000030300000382020E1
:1011E00020202020221E0000000302020272120AA8
:1011F0001612227700000000000E080808080808F0
:101200000808083E0000000000000000007F9292E5
:10121000929292B70000000000000000003B46429E
:10122000424242E70000000000000000003C424251
:101230004242423C0000000000000000001B264229
:101240004242221E020700000000000000784442D3
:101250004242447840E000000000000000774C0467
:101260000404041F0000000000000000007C420293
:101270003C40423E0000000000000008083E080814
:10128000080808300000000000000000006342422F
:10129000424262DC000000000000000000E742243F
:1012A00024140808000000000000000000EB494979
:1012B000555522220000000000000000007624188E
:1012C0001818246E000000000000000000E742240F
:1012D000241418080807000000000000007E2210F7
:1012E0000808447E000000C020202020201020207C
:1012F00020202020C000101010101010101010100E
:10130000101010101010000608080808081008082F
:101310000808080806000C32C200000000000000A7
:10132000000000000000000048130008000000203A
:10133000780300006C010008F01400087803002016
:1013400028090000C801000811D40E27072A8004CC
:10135000FA0104080D1A1080010CF0FFFF0F308015
:1013600001040419246A070C091248091004011326
:101370001A011914FFFF011A03082904E90C33812B
:10138000812A0304261CFCFFFF3F1A400B5AC02889
:101390002AC00C49041BFFFF4C22411A0468230E8B
:1013A000711B07815A14010760100B010E18980178
:1013B0001C04E001181927F11A08C4231F304A0C35
:1013C000046809100C30FE3F0C30041069041BC087
:1013D0000C281E0D3030060E049C0C3010044B18E7
:1013E0008604101208060D300C860D3006EE0F3004
:1013F00002FC0D30015B0CF040193C2A0F081A105A
:101400009ED1299019CB4908890417E0FFFF03609A
:10141000C009130409161C59181A010429441A0892
:10142000045A100419F8130138041780FF1F26030B
:10143000C0FFFF071A8004293D326032181A0C13CE
:101440005A030419A41C800108045E1CFCFFFF3F22
:10145000100928041AFC0432E062405A80026DFC34
:101460001F841002290C69184DF80F080804128017
:1014700023FF7F290C490E2D8410A22045280FFE42
:101480003F0220F22702200220FA2F2221022809FF
:10149000122912290A2E02201AC95E9908165080B4
:1014A000408040195213FE1F120812042C028001C2
:1014B00062697829021AA0A518161008B8080F0941
:1014C00008090808BF0808091C092C080A78CA116D
:1014D00079012A04023CC87F3F08180BA83F182155
:1014E0000C110B12080A0E06100A8A116460000023
:0400000508000131BD
:00000001FF
